S31508000000E82B002069020008E52100089B1D00086E
S31508000010E121000809070008E94E00080000000071
S31508000020000000000000000000000000094A000867
S315080000301507000800000000750600089102000870
S31508000040930200089302000893020008930200082E
S31508000050930200089302000893020008930200081E
S31508000060930200089302000893020008930200080E
S3150800007093020008930200089302000893020008FE
S3150800008093020008930200089302000893020008EE
S3150800009093020008930200089302000893020008DE
S315080000A093020008930200089302000893020008CE
S315080000B093020008930200089302000893020008BE
S315080000C093020008930200089302000893020008AE
S315080000D093020008930200081D4E000893020008C8
S315080000E0930200089302000893020008930200088E
S315080000F0930200089302000893020008930200087E
S31508000100930200089302000893020008930200086D
S31508000110930200089302000893020008930200085D
S31508000120930200089302000893020008930200084D
S31508000130930200089302000893020008930200083D
S31508000140930200089302000893020008930200082D
S31508000150930200089302000893020008930200081D
S31508000160930200089302000893020008930200080D
S31508000170930200089302000893020008000000009A
S31508000180930200089302000800F002F800F05CF8F9
S315080001900AA090E8000C82448344AAF10107DA45D4
S315080001A001D100F051F8AFF2090EBAE80F0013F0CA
S315080001B0010F18BFFB1A43F001031847A0580000A7
S315080001C0C05800000A444FF0000C10F8013B13F029
S315080001D0070408BF10F8014B1D1108BF10F8015B92
S315080001E0641E05D010F8016B641E01F8016BF9D185
S315080001F013F0080F1EBF10F8014BAD1C0C1B09D1DC
S315080002006D1E58BF01F801CBFAD505E014F8016B4D
S3150800021001F8016B6D1EF9D59142D6D370470000DF
S315080002200023002400250026103A28BF78C1FBD8F1
S31508000230520728BF30C148BF0B6070471FB505F08D
S31508000240FBFA1FBD10B510BD00F09EF91146FFF769
S31508000250F5FF05F0BDF900F0BCF903B4FFF7F2FFAE
S3150800026003BC05F01BF80000DFF83400016841F410
S3150800027070010160BFF34F8F0A4880470A4800475C
S31508000280FEE7FEE7FEE7FEE7FEE7FEE7FEE7FEE738
S31508000290FEE7FEE705480649044A064B7047000094
S315080002A088ED00E00D4A000889010008E8270020CB
S315080002B0E82B0020E827002072B6704762B6704720
S315080002C072B602B4EFF3118180F31188BFF34F8F32
S315080002D0BFF36F8F084602BC62B6704772B680F3EA
S315080002E01188BFF34F8FBFF36F8F62B6704730BF69
S315080002F0704720BF7047B0FA80F0704790FAA0F0B8
S31508000300B0FA80F0704790FAA0F07047704753EA49
S31508000310020C00F069802DE9F04B4FF00006002B27
S315080003201FBFB3FA83F503FA05F424FA05F65E400F
S3150800033012BF1643B2FA82F502FA05F4C5F1200592
S315080003401EBF22FA05FC44EA0C04203556EA044C82
S315080003504FEA144418BF641C4FF000084FF0000918
S31508000360904271EB030C39D3002919BFB1FA81F712
S3150800037001FA07F6B0FA80F700FA07F6C7F1200780
S315080003801EBF20FA07FC46EA0C062037B6FBF4FC2B
S31508000390A7EB0507103F07F01F0BCBF120060CFA59
S315080003A00BFB2CFA06F644BFB3460026202FA4BF43
S315080003B05E464FF0000B5BEA060C08BF4FF0010BD8
S315080003C019EB0B09ABFB027C48EB0608C01B06FBC6
S315080003D002CC0BFB03CC71EB0C01C1E70B460246C2
S315080003E041464846BDE8F08B13B54FF000004FF084
S315080003F00001AFF30080BDE81C40704740EA0103E6
S31508000400024630B59B0710D14FF0013400E008C210
S3150800041008C91D1B9D4315EAC41FF8D013F0FF0138
S3150800042002F8011B0DD01B0AF8E711F8013B002B57
S3150800043002F8013B05D011F8013B002B02F8013BFD
S31508000440F3D130BD032A40F2308010F0030C00F0DF
S31508000450158011F8013BBCF1020F624498BF11F8F0
S3150800046001CB00F8013B38BF11F8013BA2F10402A9
S3150800047098BF00F801CB38BF00F8013B11F0030321
S3150800048000F05080083AC0F0088051F8043B083A5A
S3150800049051F804CBA0E80810F5E7121D5CBF51F827
S315080004A0043B40F8043BAFF30080D20724BF11F8A1
S315080004B0013B11F801CB48BF11F8012B24BF00F806
S315080004C0013B00F801CB48BF00F8012B70474FF0FD
S315080004D0000200B5134694469646203922BFA0E886
S315080004E00C50A0E80C50B1F12001BFF4F7AF090792
S315080004F028BFA0E80C5048BF0CC05DF804EB890083
S3150800050028BF40F8042B08BF704748BF20F8022BC5
S3150800051011F0804F18BF00F8012B704770477047DD
S315080005207047704710B5203AC0F00B80B1E81850F4
S31508000530203AA0E81850B1E81850A0E81850BFF4BF
S31508000540F5AF5FEA027C24BFB1E81850A0E818505E
S3150800055044BF18C918C0BDE810405FEA827C24BFB2
S3150800056051F8043B40F8043B08BF7047D20728BF40
S3150800057031F8023B48BF11F8012B28BF20F8023B8F
S3150800058048BF00F8012B7047754600F02BF8AE46B9
S3150800059005006946534620F00700854618B020B581
S315080005A0FFF778FEBDE820404FF000064FF0000741
S315080005B04FF000084FF0000B21F00701AC46ACE8FD
S315080005C0C009ACE8C009ACE8C009ACE8C0098D466A
S315080005D0704710B50446AFF300802046BDE81040CA
S315080005E0FFF73BBE004870478827002072B64EF6D4
S315080005F02250CEF2000040F2FF01C0F20001017065
S31508000600002080F3098841F27C00C2F200000168EC
S3150800061081F3088802F082FC41F2AA00C2F20000C7
S3150800062041F2AB01C2F200010A78027041F22410CD
S31508000630C2F2000041F22811C2F200010A68026003
S31508000640106880F30988EFF3148040F0020020F068
S31508000650040080F31488BFF36F8FBDE8F04F0FBC1A
S31508000660BDE8005006BC62B6084726484FF08051E0
S315080006700160704772B641F28002C2F20002116848
S3150800068081F31188BFF34F8FBFF36F8F62B6EFF315
S3150800069009801EF0100F08BF20ED108A20E9F04FE0
S315080006A041F22415C2F2000529680860744602F072
S315080006B035FC41F2AA00C2F2000041F2AB01C2F2D7
S315080006C000010A78027041F22811C2F200010A6894
S315080006D02A6044F0040E1068B0E8F04F1EF0100FC0
S315080006E008BFB0EC108A80F3098840F20002C0F215
S315080006F0000272B682F31188BFF34F8FBFF36F8F74
S3150800070062B6704704ED00E000BFFEE700BFFEE7F3
S3150800071000207047704710B5024692F82030012B2A
S3150800072001D0022B1CD101F0010028B110688068A5
S3150800073040F080001468A06001F0020028B110683B
S31508000740806840F400401468A06001F0040028B1F5
S315080007501068806840F400001468A060002010BD8E
S31508000760506A40F4802050620120F8E7F0B504464C
S315080007700D461E4694F8207020688368A86800B95C
S3150800078000E000BF012F01D0022F7CD103F080606A
S3150800079030B903F0006018B903F08050002873D010
S315080007A0C3F30161022905D9606A40F4000060625A
S315080007B00120F0BD012088403060A86860B9B5F80E
S315080007C000C0E86840EA4C5C206800F5C07000EBA1
S315080007D00110C0F800C00FE0D5E901C040EACC001E
S315080007E0D5F80CC040EA0C00D4F800C00CF5C07C63
S315080007F00CEB011CCCF80000D5F810C0206800F5F9
S31508000800C07000EB0110C0F804C0287D01280ED185
S31508000810206800F5C07000EB0110406840F4807C49
S31508000820206800F5C07000EB0110C0F804C0D0794C
S31508000830000692F806C040EA0C4092F805C040EA65
S315080008400C2C10794CEA000C206800F5C07000EBFF
S315080008500110C0F80CC0D078000692F802C040EA31
S315080008600C4092F801C040EA0C2092F800C040EA19
S315080008700C00D4F800C00CF5C07C0CEB011CCCF8BD
S315080008800800206801E016E00FE000F5C07000EBF4
S315080008900110006840F0010C206800F5C07000EBFC
S315080008A00110C0F800C0002083E7606A40F4001019
S315080008B0606201207DE7606A40F480206062012062
S315080008C077E70000F0B504460A46216894F82050F8
S315080008D0012D01D0022D7ED1424901F5007108682B
S315080008E040F001000860086820F47C500860086839
S315080008F0566A40EA06200860107D00F01F060120AF
S3150800090000FA06F3C8699843C861A1F50071D06971
S31508000910C8B9D1F80C029843C1F80C02908880B285
S31508000920968940EA064601F51070576940F837601F
S31508000930108880B2168940EA064601F51070576994
S3150800094000EBC7004660D069012819D1D1F80C021E
S315080009501843C1F80C02908880B2168840EA064609
S3150800096001F51070576940F83760908980B216898A
S3150800097040EA064601F51070576900EBC700466065
S31508000980906928B9D1F804029843C1F8040204E032
S31508000990D1F804021843C1F80402106928B9D1F83D
S315080009A014029843C1F8140204E0D1F8140218435B
S315080009B0C1F81402106A012804D1D1F81C021843A0
S315080009C0C1F81C02D1F8000220F00100C1F80002AB
S315080009D00020F0BDFFE7606A40F4802060620120D5
S315080009E0F7E700000064004010B50246002092F8C0
S315080009F02030012B01D0022B09D121B91468E468F3
S31508000A0004F0030003E01468246904F0030010BD31
S31508000A1070B5044694F82050012D01D0022D7DD1E1
S31508000A2051B92068C06800F0030080B9606A40F4D4
S31508000A3000106062012070BD2068006900F00300A4
S31508000A4028B9606A40F4001060620120F3E7206864
S31508000A5000F5D87000EB0110006800F00400906003
S31508000A60906840B9206800F5D87000EB011000685E
S31508000A70400D106007E0206800F5D87000EB011003
S31508000A800068C0085060206800F5D87000EB0110B7
S31508000A90006800F00200D060206800F5D87000EB0E
S31508000AA00110406800F00F001061206800F5D8704A
S31508000AB000EB0110406800F47F40000A906120684E
S31508000AC000F5D87000EB01104068000C50612068F2
S31508000AD000F5D87000EB011080681870206800F5E2
S31508000AE0D87000EB0110806800F47F40000A587047
S31508000AF0206800F5D87000EB0110806800F47F00CC
S31508000B00000C9870206800F5D87000EB011080681A
S31508000B10000ED870206800F5D87000E02FE000EBD2
S31508000B200110C0681871206800F5D87000EB011034
S31508000B30C06800F47F40000A5871206800F5D87034
S31508000B4000EB0110C06800F47F00000C9871206863
S31508000B5000F5D87000EB0110C068000ED87131B9E5
S31508000B602068C06840F020002668F06005E020682C
S31508000B70006940F020002668306100205BE7606A63
S31508000B8040F480206062012055E70146002091F874
S31508000B902020012A01D0022A11D10B689B6803F094
S31508000BA0806303B1401C0B689B6803F0006303B1C4
S31508000BB0401C0B689B6803F0805303B1401C7047C8
S31508000BC070B504460CB9012070BD94F8200010B920
S31508000BD0204600F0AFF82068006820F0020021687F
S31508000BE0086000F0A7FA05460DE000F0A3FA401BDE
S31508000BF00A2808D9606A40F400306062052084F843
S31508000C0020000120E0E72068406800F00200002884
S31508000C10EBD12068006840F001002168086000F008
S31508000C2089FA05460DE000F085FA401B0A2808D91E
S31508000C30606A40F400306062052084F820000120D4
S31508000C40C2E72068406800F001000028EBD0207E4B
S31508000C50012806D12068006840F0800021680860F5
S31508000C6005E02068006820F0800021680860607E42
S31508000C70012806D12068006840F040002168086015
S31508000C8005E02068006820F0400021680860A07E22
S31508000C90012806D12068006840F020002168086015
S31508000CA005E02068006820F0200021680860E07EE2
S31508000CB0012806D12068006820F010002168086025
S31508000CC005E02068006840F0100021680860207F71
S31508000CD0012806D12068006840F0080021680860ED
S31508000CE005E02068006820F0080021680860607F39
S31508000CF0012806D12068006840F0040021680860D1
S31508000D0005E02068006820F0040021680860D4E93E
S31508000D100201084321690843616908436168491E5D
S31508000D2008432168C86100206062012084F8200019
S31508000D30002049E710B586B004462849206888424D
S31508000D404AD100BF00BF002000902548006840F047
S31508000D500100234908600846006800F00100009079
S31508000D6000BF00BF00BF00BF00BF002000900846BC
S31508000D70006840F0010008600846006800F00100BD
S31508000D80009000BF00BF00BF00BF002000901448BD
S31508000D901030006840F000701149103108600846AC
S31508000DA0006800F00070009000BF00BF8814019032
S31508000DB00220029001200390022004900920059049
S31508000DC001A9084800F0A8F84FF40060019001A9AD
S31508000DD0044800F0A1F800BF06B010BD006400404A
S31508000DE0303802400000024070B5044694F82000EE
S31508000DF0012822D1022084F820002068006820F00B
S31508000E0001002168086000F095F905460DE000F03C
S31508000E1091F9401B0A2808D9606A40F400306062DC
S31508000E20052084F82000012070BD2068406800F085
S31508000E3001000028EBD16062F6E7606A40F4002002
S31508000E4060620120F0E770B50446A56D00F072F9FE
S31508000E50064694F83500022808D08020606500BF51
S31508000E60002084F8340000BF012070BD20680068A7
S31508000E7020F01600216808602068406920F080008C
S31508000E8021684861206C08B9A06C28B12068006800
S31508000E9020F00800216808602068006820F001003A
S31508000EA0216808600FE000F045F9801B05280AD97B
S31508000EB02020606500BF002084F8340000BF0320AE
S31508000EC084F83500D1E72068006800F001000028A2
S31508000ED0E9D194F85C103F208840A86000BF002044
S31508000EE084F8340000BF012084F835000020BCE7F0
S31508000EF0014691F83500022803D080204865012074
S31508000F007047052081F835000868006820F0010060
S31508000F100A6810600020F3E7F8B502460B4600257C
S31508000F20002400200021DEE0012606FA01F51E68ED
S31508000F3006EA0504AC4275D11E7906F00306012EB1
S31508000F4004D01E7906F00306022E13D190684F00CE
S31508000F500326BE40B0434F00DE68BE403043906073
S31508000F60506801268E40B0431E79C6F300168E409F
S31508000F70304350601E7906F00306032E09D0D06868
S31508000F804F000326BE40B0434F009E68BE40304324
S31508000F90D0601E7906F00306022E13D1CF0802F19F
S31508000FA0200656F827004E07F70E0F26BE40B04318
S31508000FB04F07FF0E1E69BE403043CF0802F12006D8
S31508000FC046F8270010684F000326BE40B0431E7936
S31508000FD006F003064F00BE40304310605E6806F018
S31508000FE08056B6F1805F7DD100BF00260096404E40
S31508000FF0366846F480463E4F3E603E46366806F4FE
S315080010008046009600BF00BF3A4E8F0856F8270064
S315080010108E07370F0F26BE40B043374EB24202D175
S31508001020002624E05EE0354EB24201D101261EE0DC
S31508001030334EB24201D1022619E0324EB24201D1F4
S31508001040032614E0304EB24201D104260FE02F4E9B
S31508001050B24201D105260AE02D4EB24201D106263A
S3150800106005E02C4EB24201D1072600E008268F077C
S315080010703F0FBE4030431F4E8F0846F82700264EC6
S315080010803068A0435E6806F48036B6F5803F00D126
S315080010902043214E3060361D3068A0435E6806F452
S315080010A00036B6F5003F00D120431B4E361D306092
S315080010B0361D3068A0435E6806F48016B6F5801FB4
S315080010C000D12043144E08363060361D3068A043E0
S315080010D05E6806F40016B6F5001F00D120430E4ED2
S315080010E00C363060491C1029FFF41EAFF8BD00000D
S315080010F0443802400838014000000240000402401B
S3150800110000080240000C0240001002400014024091
S3150800111000180240001C0240003C01400AB18161EF
S3150800112001E00B048361704701480068000C7047B2
S31508001130002004E001480068704700006C10002099
S3150800114010B50A48006840F4007008490860084667
S31508001150006840F480600860032000F07FF80F20E4
S3150800116000F006F800F02AF8002010BD003C024006
S3150800117070B504460E4800784FF47A71B1FBF0F06A
S315080011800C490968B1FBF0F5284600F01DFC08B1CA
S31508001190012070BD102C07D200222146501E00F0F7
S315080011A01EF80548046001E00120F2E70020F0E798
S315080011B07410002078100020701000207047014637
S315080011C00846002809DB00F01F0301229A4043095C
S315080011D09B0003F1E023C3F8002100BF70472DE907
S315080011E0F05F80460D461646002704F03BF8074692
S315080011F039462A46334601F00700C0F1070ABAF114
S31508001200040F02D94FF0040A01E0C0F1070AD146DB
S3150800121000F1040ABAF1070F02D24FF0000A01E002
S31508001220A0F1030AD4464FF0010A0AFA09FAAAF10C
S31508001230010A0AEA020A0AFA0CFA4FF0010B0BFA3B
S315080012400CFBABF1010B0BEA030B4AEA0B04214634
S31508001250404604F00FF8BDE8F09F000000BF00F01C
S315080012600702064B19684FF6FF031940044B0B4358
S3150800127043EA0221014B196000BF70470CED00E0FC
S315080012800000FA0570B504460D460CB9012070BD7C
S315080012905848006800F00700A84209D255490D7061
S315080012A00846006800F00700A84201D00120EEE7D2
S315080012B0207800F0020002281DD1207800F00400F2
S315080012C0042805D14C48006840F4E0504A490860B3
S315080012D0207800F00800082805D14748006840F43F
S315080012E06040454908604448006820F0F000A1685D
S315080012F0084341490860207800F00100A8B36068F7
S31508001300012807D13C4808380068C0F34040B8B9FE
S315080013100120BCE76068022802D06068032807D16C
S31508001320354808380068C0F3406048B90120AEE780
S31508001330314808380068C0F3400008B90120A6E71C
S315080013402D48006820F00300616808432A490860B0
S31508001350FFF7F0FE064609E0FFF7ECFE801B41F2B8
S315080013608831884202D9032091E707E022480068BD
S3150800137000F00C006168B0EB810FEDD11D480068E4
S3150800138000F00700A84209D91A490D7008460068F6
S3150800139000F00700A84201D0012078E7207800F085
S315080013A00400042807D11448006820F4E050E168D6
S315080013B0084311490860207800F00800082808D179
S315080013C00D48006820F46040216940EAC1000A49D6
S315080013D0086000F03FF808490968C1F30311074A95
S315080013E0515CC8400649086006480068FFF7C0FE19
S315080013F000204CE7003C02400838024068580008C4
S31508001400781000207010002001480068704700001E
S315080014107810002000B5FFF7F7FF04490968C1F303
S315080014208221034A515CC84000BD000008380240CA
S315080014307858000800B5FFF7E7FF04490968C1F3C3
S315080014404231034A515CC84000BD000008380240DA
S31508001450785800082DE9F047002400250026A14603
S315080014602548006800F00C0020B1042805D008289B
S315080014703AD105E0DFF8849039E0DFF8849036E069
S315080014801D48001F006800F03F041B48001F006845
S3150800149000F4800078B11A481749091F0968C1F392
S315080014A08811A0FB01700146224600233846FEF744
S315080014B02EFF05460EE011480F49091F0968C1F3BA
S315080014C08811A0FB01700146224600233846FEF724
S315080014D01EFF05460848001F0068C0F30140401C6F
S315080014E04600B5FBF6F902E0DFF8109000BF00BF32
S315080014F04846BDE8F0870000083802400024F4009A
S3150800150000127A00F8B504460CB90120F8BD207817
S3150800151000F00100002874D0F948006800F00C00BB
S3150800152004280DD0F648006800F00C00082813D1EE
S31508001530F348001F006800F48000B0F5800F0BD157
S31508001540EF4808380068C0F34040002859D0606862
S31508001550002856D10120D9E700BF6068B0F5803F62
S3150800156008D1E7480838006840F48030E44908396B
S3150800157008601EE06068B0F5A02F0DD1E048083875
S31508001580006840F48020DE4908390860084600688B
S3150800159040F4803008600CE0D9480838006820F428
S315080015A08030D749083908600846006820F480204A
S315080015B0086000BF606890B1FFF7BCFD054606E00D
S315080015C0FFF7B8FD401B642801D903209EE7CC48E5
S315080015D008380068C0F340400028F1D011E0FFF752
S315080015E0A9FD054606E0FFF7A5FD401B642801D9BD
S315080015F003208BE7C24808380068C0F3404000283B
S31508001600F1D1207800F0020002285FD1BC480068BA
S3150800161000F00C0058B1BA48006800F00C00082821
S315080016201CD1B748001F006800F48000B0B9B44860
S3150800163008380068C0F3400020B1E068012801D0EE
S31508001640012063E7AE480838006820F0F8002169F1
S3150800165040EAC100AA490839086037E0E06800B3E3
S315080016600120A8490860FFF765FD054606E0FFF773
S3150800167061FD401B022801D9032047E7A048083826
S315080016800068C0F340000028F1D09D48083800687B
S3150800169020F0F800216940EAC10099490839086034
S315080016A014E0002097490860FFF744FD054606E068
S315080016B0FFF740FD401B022801D9032026E7904882
S315080016C008380068C0F340000028F1D1207800F0FF
S315080016D0080008282CD16069A8B101208A49086049
S315080016E0FFF728FD054606E0FFF724FD401B022804
S315080016F001D903200AE782486C300068C0F340002D
S315080017000028F1D014E000207F490860FFF712FD99
S31508001710054606E0FFF70EFD401B022801D9032007
S31508001720F4E677486C300068C0F340000028F1D131
S31508001730207800F00400042870D10027704838305B
S31508001740006800F0805090B900BF002000906C48F7
S315080017503830006840F080506949383108600846DA
S31508001760006800F08050009000BF00BF012767485E
S31508001770006800F48070B0B96448006840F480706E
S3150800178062490860FFF7D6FC054606E0FFF7D2FC7B
S31508001790401B022801D90320B8E65C48006800F41B
S315080017A080700028F2D000BFA068012808D15448EC
S315080017B06830006840F001005149683108601DE052
S315080017C0A06805280DD14E486830006840F004002E
S315080017D04B49683108600846006840F00100086017
S315080017E00CE047486830006820F001004449683139
S315080017F008600846006820F00400086000BFA0687A
S31508001800A8B1FFF797FC054609E0FFF793FC401BD4
S3150800181041F28831884202D9032077E626E0384823
S3150800182068300068C0F340000028EED013E0FFF7E8
S3150800183081FC054608E0FFF77DFC401B41F2883134
S31508001840884201D9032061E62D4868300068C0F354
S3150800185040000028EFD1012F07D129483830006809
S3150800186020F0805026493831086000BFA06900285A
S3150800187045D02348006800F00C0008285DD0A06910
S31508001880022845D100201F490866FFF753FC054684
S3150800189006E0FFF74FFC401B022801D9032035E676
S315080018A0174808380068C0F340600028F1D1D4E929
S315080018B007010843616A40EA81110122A06AC2EB66
S315080018C0500041EA00412C20005D41EA00600C49C5
S315080018D0091F086001200B490866FFF72BFC05461F
S315080018E006E0FFF727FC401B022801D903200DE676
S315080018F0034808380068C0F340600028F1D049E082
S315080019000838024000004742800E474200700040F7
S31508001910002021490866FFF70DFC054606E0FFF79B
S3150800192009FC401B022801D90320EFE51B48006883
S31508001930C0F340600028F2D12CE0A069012800D14C
S31508001940E4E51648001D0668A069012820D006F4BB
S315080019508001E06981421BD106F03F01206A81427D
S3150800196016D147F6C0703040616AB0EB811F0FD1BF
S3150800197006F440310122A06AC2EB5000B1EB004FD9
S3150800198006D106F070612C20005DB1EB006F01D026
S315080019900120BBE50020B9E50000474200380240B7
S315080019A0042808D14FF0E021096941F004014FF0FD
S315080019B0E022116107E04FF0E021096921F00401F6
S315080019C04FF0E0221161704770B504462546681E3F
S315080019D0B0F1807F01D301200FE0681E4FF0E021AF
S315080019E048610F214FF0FF3003F044FC00204FF010
S315080019F0E021886107200861002070BD70477047A4
S31508001A0001460022002391F83D2091F83E3042EA33
S31508001A10030070472DE9F84F0446206805682068DA
S31508001A20C668206847694FF00009CA4605F00F09DD
S31508001A30B9F1000F0AD105F0200038B106F02000F0
S31508001A4020B1204603F021F8BDE8F88FB9F1000F60
S31508001A5072D007F0010018B906F4907000286BD010
S31508001A6005F0010030B106F4807018B1206C40F022
S31508001A700100206405F0040030B107F0010018B138
S31508001A80206C40F00200206405F0020030B107F037
S31508001A90010018B1206C40F00400206405F008002D
S31508001AA048B106F0200010B907F0010018B1206C03
S31508001AB040F008002064206C70B305F0200028B1BF
S31508001AC006F0200010B1204602F0DFFF20684069CA
S31508001AD0C0F3801A206C00F0080010B9BAF1000FA4
S31508001AE023D0204602F0A6FF2068406900F0400097
S31508001AF0402816D12068406920F0400021684861D6
S31508001B00A06B50B15648A16B0865A06BFFF7F0F9BA
S31508001B1010B1A06B016D88470CE02046FFF76FFFF8
S31508001B2008E02046FFF76BFF04E02046FFF767FF53
S31508001B300020206488E7FFE7206B012879D105F0AB
S31508001B401000002875D006F01000002871D000BFDC
S31508001B500020009020680068009020684068009087
S31508001B6000BF00BF2068406900F04000402839D116
S31508001B70A06B006840681FFA80F8B8F1000F30D0F3
S31508001B80A08D40452DDDA4F82E80A06BC069B0F568
S31508001B90807F1FD02068C06820F480702168C860E4
S31508001BA02068406920F00100216848612068406982
S31508001BB020F0400021684861202084F83E0000207B
S31508001BC020632068C06820F010002168C860A06BF8
S31508001BD0FFF739F9A08DE28D801A81B22046FFF70A
S31508001BE00DFF31E7A08DE18D401A1FFA80F8E08DD0
S31508001BF0E8B1B8F1000F1AD02068C06820F49070D8
S31508001C002168C8602068406920F0010021684861A1
S31508001C10202084F83E00002020632068C06820F059
S31508001C2010002168C86041462046FFF7E7FE0BE72B
S31508001C30FFE705F0800030B106F0800018B12046B5
S31508001C4003F0BBF800E705F0400030B106F04000AD
S31508001C5018B1204602F009FFF6E600BFF4E60000D8
S31508001C60214A000810B504460CB9012010BDA06928
S31508001C7000B100E000BF94F83D0028B9002084F8C0
S31508001C803C00204600F027F8242084F83D00206810
S31508001C90C06820F400502168C860204602F054FF4E
S31508001CA02068006920F4904021680861206840692E
S31508001CB020F02A00216848612068C06840F4005076
S31508001CC02168C86000202064202084F83D0084F83C
S31508001CD03E000020CAE7704770B504460D46164612
S31508001CE094F83E00202816D105B10EB9012070BD22
S31508001CF000BF94F83C00012801D10220F7E7012033
S31508001D0084F83C0000BF002020633246294620465E
S31508001D1003F030F8EBE70220E9E700001B490988E1
S31508001D2001F4004189BB1949098801F4804171B160
S31508001D30174909780A2903D00021144A118024E09A
S31508001D401249098841F40041104A11801DE01049E2
S31508001D5009780D2906D10D49098841F480410B4AB5
S31508001D60118012E00A490978084A1288C2F30D025E
S31508001D70084B995405490988491C044A118011469B
S31508001D800988C72901DD0021118070475C0E0020F3
S31508001D905E0E00202C110020704700BFFEE70000F1
S31508001DA010B586B000BF002000905948006840F082
S31508001DB00100574908600846006800F001000090D5
S31508001DC000BF00BF00BF002000900846006840F032
S31508001DD0020008600846006800F00200009000BF94
S31508001DE000BF00BF002000900846006840F00400CD
S31508001DF008600846006800F00400009000BF00BFB5
S31508001E0000BF002000900846006840F08000086087
S31508001E100846006800F08000009000BF00BF00BFC1
S31508001E20002000900846006840F008000860084650
S31508001E30006800F00800009000BF00BF00BF002047
S31508001E4000900846006840F01000086008460068E0
S31508001E5000F01000009000BF00BF00BF00200090F7
S31508001E600846006840F0200008600846006800F050
S31508001E702000009000BF00BF00BF00200090084669
S31508001E80006840F4807008600846006800F48070B6
S31508001E90009000BF00BF00BF002000900846006801
S31508001EA040F0400008600846006800F040000090D6
S31508001EB000BF00BF002427E004EB4400154901EBEE
S31508001EC0C0008088019004EB440001EBC0008068E4
S31508001ED0029004EB440001EBC000C068039004EBD9
S31508001EE0440001EBC0000069049004EB440001EBD8
S31508001EF0C0004069059004EB4401064A52F83100D7
S31508001F0001A9FFF709F8641C102CD5D306B010BD3B
S31508001F1030380240E80E002030B587B00546142157
S31508001F2002A8FEF7D4FA00BF00200190A148006875
S31508001F3040F010009F4908600846006800F010004D
S31508001F40019000BF00BF00BF00200190081F006875
S31508001F5040F40030091F08600846006800F40030A5
S31508001F60019000BF00BF00BF00200190084600682E
S31508001F7040F4802008600846006800F4802001903C
S31508001F8000BF00BF00BF002001900846006840F46B
S31508001F90002008600846006800F40020019000BF91
S31508001FA000BF00BF0020019082481438006840F046
S31508001FB001008049143908600846006800F00100ED
S31508001FC0019000BF00BF00BF0020019008460068CE
S31508001FD040F0080008600846006800F00800019014
S31508001FE000BF00BF0024CEE004EB440000EBC400B1
S31508001FF0714901EB800000890290022003900020BD
S315080020000490032005900720069004EB440101EB99
S31508002010C401694A02EB8101486802A9FEF77CFF00
S3150800202004EB440000EBC400634901EB8000008A1E
S3150800203002900720069004EB440101EBC4015E4AB6
S3150800204002EB8101C86802A9FEF766FF04EB4400AB
S3150800205000EBC400584951F8200004EB0411574A14
S3150800206042F8210004EB0410114601EB800045609C
S3150800207004EB440000EBC4004F4901EB80004169C2
S3150800208004EB041002EB8000816004EB440000EBD3
S31508002090C400494901EB8000816904EB041002EB96
S315080020A08000C16004EB440000EBC400424901EB28
S315080020B08000C16904EB041002EB8000016104EBA7
S315080020C0440000EBC4003C4901EB8000016A04EBC4
S315080020D0041002EB8000416104EB440000EBC400ED
S315080020E0354901EB8000416A04EB041002EB8000DD
S315080020F0816104EB440000EBC4002F4901EB80002A
S31508002100816A04EB041002EB8000C16104EB041140
S3150800211002EB8100FFF7A6FD04EB440000EBC400C8
S31508002120254951F820002649884207D10122032172
S315080021302520FFF754F82520FFF741F804EB440063
S3150800214000EBC4001C4951F820001E49884207D1FB
S31508002150022203212720FFF742F82720FFF72FF84E
S3150800216004EB440000EBC400134951F8200016495B
S31508002170884207D1032211463420FFF730F834206D
S31508002180FFF71DF8641C032CFFF42EAF0F480288D6
S315080021900F491048FFF7A0FD0C4802880C490E4865
S315080021A0FFF79AFD0948028809490C48FFF794FD8C
S315080021B007B030BD44380240640E0020C01200202B
S315080021C00010014000480040004C0040600E00200E
S315080021D05E0E0020F4110020381200207C12002028
S315080021E000BFFEE77047704770B5044600F09EF8DA
S315080021F00020394908703949087039490870394941
S3150800220008603949086039490870394908703949F8
S315080022100870394800680A21B0FBF1F037490860B0
S315080022203748056845B13748066803E0761E00203A
S3150800223028602D1D002EF9D1324801683048006803
S3150800224001F0B0FE01F094FA01F0B6FA00202E492A
S3150800225008602E490880204601F07CF8208800B1E5
S3150800226070BD204601F082F8208800B1F8E700200A
S3150800227027490860274908802749086027490880B0
S315080022802749086027490880204601F005FE20886E
S3150800229000B1E5E7204601F025F8208800B1DFE720
S315080022A0204601F08BFE208800B1D9E7204601F0D0
S315080022B0BFFC208800B1D3E7204602F041F8208809
S315080022C000B1CDE700F0D6FEFFF78DFF01201649D5
S315080022D0087000BFC4E7000088100020891000209D
S315080022E0B61000202411002028110020AA10002072
S315080022F0AB100020BC100020D4580008B8100020ED
S31508002300A0580008A458000894100020981000202F
S31508002310A4100020A8100020B0100020B41000203F
S31508002320C0100020C41000208A1000200C4909683B
S315080023300C4A126801EB82010B4A116011460968C2
S3150800234021F0070111600949086800F04041B1F120
S31508002350404F01D000BFFEE74021054A1160704793
S31508002360A0580008A45800087C10002034EF00E0AC
S315080023708010002070B5002538480078012800D064
S3150800238070BD00BF4020FDF79BFF054600BF3448DF
S31508002390007828B900BF2846FDF7A0FF00BFEFE781
S315080023A02F480078401E2E4908700846007828B144
S315080023B000BF2846FDF792FF00BFE1E729480078ED
S315080023C028B100BF2846FDF789FF00BFD8E7264891
S315080023D001682648006801F0D1FD0446012C02D0A8
S315080023E0002000F0ABF901F0B9F921490870084658
S315080023F0007800EB40001F4951F820001E4908608C
S31508002400084600681D49096888420FD1002000F077
S3150800241069FD0446012C03D01848006800F08EF9BF
S3150800242000BF2846FDF75AFF00BFA9E71248006813
S31508002430D0F89400401C10490968C1F89400104867
S315080024400068401C0E490860FEF70FF900BF2846D1
S31508002450FDF744FF00BF00BF92E700008910002087
S3150800246088100020B6100020A4580008A0580008BC
S31508002470AB1000202C240020281100202411002055
S31508002480E41000202DE9F04104460E4615460027C3
S315080024902148007820B142F6E1602880BDE8F08145
S315080024A01CB945F6C3502880F8E700BF00BF402096
S315080024B0FDF706FF074600BF00BF18492068884297
S315080024C00AD100BF00BF3846FDF708FF00BF00BFAE
S315080024D045F6C1502880E1E7104820606660002074
S315080024E02062606284F82800E06204F1080001F0C6
S315080024F080F8204600F0A0FF09480088401C0849DB
S31508002500088000BF00BF3846FDF7E8FE00BF00BFE1
S315080025100020288000BFC1E7881000204D55545878
S31508002520A81000202DE9F0470646894617461C469E
S31508002530089D4FF0000A7C48007820B146F2AE109C
S315080025402880BDE8F08779480078012803D045F649
S3150800255089602880F5E71EB945F6C3502880F0E75C
S315080025601FB1B7F5004F02D100E000BF03E045F602
S3150800257025602880E5E700BF6D493068884203D0AA
S3150800258045F6C4502880DCE700BF00BF4020FDF7B1
S3150800259097FE824600BF00BF96F82800B8B965487E
S315080025A000687062012086F828000CB1F06A206085
S315080025B031466048006800F057FF00BF00BF50462C
S315080025C0FDF78CFE00BF00BF00202880B9E75949F7
S315080025D0706A0968884221D196F82800FF280AD12E
S315080025E000BF00BF5046FDF779FE00BF00BF45F2A9
S315080025F084702880A5E796F82800401C86F82800ED
S315080026000CB1F06A206000BF00BF5046FDF766FEB9
S3150800261000BF00BF45F28270288092E707F40040A9
S3150800262068B100BF00BF5046FDF758FE00BF00BFA7
S315080026300CB10020206046F2B010288081E73E48A1
S31508002640007868B100BF00BF5046FDF747FE00BFDF
S3150800265000BF0CB10020206046F66350288070E762
S31508002660D6F8248098F83B003249096891F83B105F
S31508002670884206DD2F48006890F83B10404601F076
S315080026805DFB4B4604222B480168304600F042FFAA
S3150800269000BF00BF5046FDF721FE00BF00BF00F097
S315080026A055F800BF00BF4020FDF70AFE824600BF6E
S315080026B000BF2048006890F8390030B101280CD0D6
S315080026C002281AD0032821D110E01CB11948006845
S315080026D0C06C2060002028801CE01CB115480068EA
S315080026E0C06C206046F2A910288013E00CB10020C7
S315080026F0206047F2D92028800CE01CB10D480068FC
S31508002700C06C206045F6C250288003E046F62E606D
S31508002710288000BF00BF00BF00BF5046FDF7DEFDA2
S3150800272000BF00BF00BF0CE78810002089100020FA
S315080027304D55545824110020B610002010B50446F3
S3150800274000BFFDF7E3FF00BF10BD000010B5002471
S3150800275022480078012800D010BD2148007800B131
S31508002760FAE72048007800B1F6E700BF4020FDF7F9
S31508002770A7FD044600BF00F0F1FF1B490870084694
S31508002780007800EB4000194951F820001849086004
S315080027900846006817490968884205D100BF2046DF
S315080027A0FDF79CFD00BFD7E711480068D0F89400F4
S315080027B0401C0F490968C1F894000F480068401C7E
S315080027C00D490860FDF751FF00BF2046FDF786FD5D
S315080027D000BFBFF36F8F00BFBEE70000891000205F
S315080027E088100020B6100020AB1000202C240020F2
S315080027F02811002024110020E410002070B504469A
S315080028001C480078012803D045F68B60208070BDEF
S3150800281000256D1C6D1C6D1C17480088A84203DC3A
S3150800282045F68C602080F2E714480078E8B900F095
S3150800283095FF134908700846007812490870104831
S31508002840007800EB4000104951F820000F49086055
S31508002850084600680E490860012008490870FDF717
S31508002860C5FE43F69920208002E045F68A6020805E
S3150800287000BFCCE78A100020EC1000208910002049
S31508002880AB100020AA1000202C24002028110020BC
S31508002890241100202DE9F04107464FF0000800BF3B
S315080028A000BF4020FDF70CFD804600BF00BF00209A
S315080028B03B4908803B4908603B4908603B4908603A
S315080028C03B4908603B4908603B49088100BF00BF97
S315080028D04046FDF703FD00BF00BF00BF00BF402014
S315080028E0FDF7EEFC804600BF00BF3448046800BF11
S315080028F000BF4046FDF7F2FC00BF00BF21E000BF65
S3150800290000BF4020FDF7DCFC804600BF00BF00206A
S3150800291044F8800FE0626061208260822062606213
S31508002920FDF7F6FEE061803C04F16C060020B081FC
S31508002930D4F8BC4000BF00BF4046FDF7CFFC00BF3F
S3150800294000BF002CDBD100BF00BF4020FDF7B8FC5C
S31508002950804600BF00BF1A48056800BF00BF404652
S31508002960FDF7BCFC00BF00BF13E000BF00BF40205E
S31508002970FDF7A6FC804600BF00BF05F12006002033
S31508002980B081AD6900BF00BF4046FDF7A7FC00BF98
S3150800299000BF002DE9D100203880BDE8F081000095
S315080029A0CA100020E0100020FC10002000110020B2
S315080029B0141100201811002020240020E8100020FF
S315080029C0B0100020704700002DE9FF4F85B004467F
S315080029D09346DDE91995DDE91286159F00200290D8
S315080029E06248007828B147F24A10288009B0BDE845
S315080029F0F08F1CB947F2AD102880F7E7BBF1000F3E
S31508002A0003D147F24F102880F0E71EB946F62F602B
S31508002A102880EBE756480068874203D246F63060BE
S31508002A202880E3E71498B84203D346F63160288035
S31508002A30DCE7B8F11E0F06D9B8F11F0F03D046F22E
S31508002A4073202880D2E7B8F11F0F06D1494884427F
S31508002A5003D046F273202880C8E7204601F02CFAF6
S31508002A600020288009F0010010B909F0020088B199
S31508002A7009F0020070B1B2460020049007E0002079
S31508002A80CAF800000AF1040A0498401C0490049845
S31508002A90B842F4D3149806EB80000390CDE9007988
S31508002AA032465846039B089900F0B4F98246B24567
S31508002AB003D246F63260288098E73946304601F058
S31508002AC071FAC4F824B00898A0620698E06084F801
S31508002AD03B8084F83C80C4F800A00398A06017984F
S31508002AE0E065179818B924480068206601E0179829
S31508002AF020661898606026626764A4F8489004F116
S31508002B006C00169900F090FC204600F03BF800BFD8
S31508002B1000BF4020FDF7D4FB029000BF00BF94F829
S31508002B203B0000F031FE204600F08EFE204601F004
S31508002B3079F912480088401C104908801048007826
S31508002B40012807D000BF00BF0298FDF7C7FB00BFEA
S31508002B5000BF4BE700BF00BF0298FDF7BFFB00BFF1
S31508002B6000BFFFF7F3FD00BF40E700008810002014
S31508002B70D05800085C230020B8100020EC10002074
S31508002B8089100020704700002DE9F04104460E46E2
S31508002B904FF000086148007820B147F24E103080A7
S31508002BA0BDE8F0815E480078012803D045F68960C3
S31508002BB03080F5E75B48844203D147F24C103080F9
S31508002BC0EEE784B900BF00BF4020FDF779FB8046D9
S31508002BD000BF00BF5448046800BF00BF4046FDF769
S31508002BE07DFB00BF00BF00BF00BF4020FDF768FBAC
S31508002BF0804600BF00BF94F83A0008285ED2DFE896
S31508002C0000F004090E10080A0F11204600F03AFEDB
S31508002C105FE05EE000BF204601F07AFA59E000BFA7
S31508002C2000BF00BF94F83800082839D2DFE800F062
S31508002C30040705380D08090600BF00BF31E000BFCC
S31508002C4000BF204600F00DFD2BE0606B456A15F8C5
S31508002C503B7F204600F005FD287869783B3D884291
S31508002C6012D095F83B0094F83B1088420CD12846C0
S31508002C7000F02DFC074695F83C00B84202DA95F8B4
S31508002C803C0000E038460746002084F8380095F8EE
S31508002C903B00B84203D03946284601F04FF800E019
S31508002CA000BF00BF94F83A00032803D094F83A000E
S31508002CB0072802D1204601F02BFA0AE000BF00BF20
S31508002CC04046FDF70BFB00BF00BF46F62D6030807F
S31508002CD066E700BF206C10B1204600F0C9FB04F17E
S31508002CE06C0000F081FB204600F022F8204601F037
S31508002CF0B1F80E480088401E0C490880FF2084F869
S31508002D003A000020308000BF00BF4046FDF7E6FAD3
S31508002D1000BF00BFFFF71AFD00BF41E7881000207B
S31508002D20891000205C23002024110020EC100020CC
S31508002D30704770472DE9F05F05460E4617461C4654
S31508002D404FF0000B3148007820B147F25910208027
S31508002D50BDE8F09F1EB946F2D5202080F8E71FB9D6
S31508002D6046F2D5202080F3E700BF00BF4020FDF7DC
S31508002D70A7FA834600BF00BF0DB92548056828682D
S31508002D8068B900BF00BF5846FDF7A8FA00BF00BFE4
S31508002D9000203060386047F252102080D8E795F856
S31508002DA0480000F0010068B900BF00BF5846FDF7AB
S31508002DB095FA00BF00BF00203060386047F2541013
S31508002DC02080C5E7D5F820A00AF1200AD5F8449056
S31508002DD000BF00BF5846FDF781FA00BF00BF4FF09D
S31508002DE0000803E00AF1040A08F10108C84503D2FD
S31508002DF0DAF800000028F5D0C6F80080A9EB08002C
S31508002E0038600020208000BFA2E70000881000205C
S31508002E1024110020F0B50446DDE9055602EB8500CD
S31508002E2020F007004FF0807C071F3846C7F800C01F
S31508002E30071F38463C60DFF8A8C0071F3846C7F8A2
S31508002E4000C04FF0123C071F3846C7F800C04FF0C5
S31508002E50033C071F3846C7F800C04FF0023C071F5F
S31508002E603846C7F800C0071F38463B60071F384674
S31508002E7039606FF0020C071F3846C7F800C04FF0DC
S31508002E80113C071F3846C7F800C04FF0103C071F13
S31508002E903846C7F800C04FF0093C071F3846C7F840
S31508002EA000C04FF0083C071F3846C7F800C04FF06F
S31508002EB0073C071F3846C7F800C04FF0063C071FF7
S31508002EC03846C7F800C04FF0053C071F3846C7F814
S31508002ED000C04FF0043C071F3846C7F800C0F0BDD5
S31508002EE0653F000830B504460CB90B480468216AEA
S31508002EF02068884206D3616C206A00EB810021684D
S31508002F00884201D8002030BD616C206A01F036F88D
S31508002F1005462846F7E700002411002070B5FDF79E
S31508002F20F7FB05461548006815490968884215D013
S31508002F3012480068D0F89C00281A10490968C1F898
S31508002F4098000E480068D0F8A0000C490968D1F826
S31508002F509810084409490968C1F8A000084800689B
S31508002F60C0F89C500020FFF7BDFF0446012C03D093
S31508002F7002480068FFF7E2FB70BD0000241100203C
S31508002F80281100202DE9F04106460D461446002773
S31508002F902748007820B147F275202080BDE8F081E7
S31508002FA024480078012803D045F689602080F5E793
S31508002FB02148007818B146F663502080EEE735B10F
S31508002FC0022D05D0042D05D0082D04D101E000BF3F
S31508002FD000BF00BF03E045F625602080DEE700BF9E
S31508002FE000BF00BF4020FDF76BF9074600BF00BFD2
S31508002FF023462A4631461148006801F043F82088DE
S3150800300038B100BF00BF3846FDF768F900BF00BFFA
S31508003010C4E70A48006800F035FC00BF00BF384620
S31508003020FDF75CF900BF00BFFFF790FB00BFB5E7EF
S315080030308810002089100020B610002024110020D6
S3150800304070B50446002600BF00BF4020FDF738F9DA
S31508003050064600BF00BF0648056800BF00BF3046E9
S31508003060FDF73CF900BF00BF00202080284670BD50
S31508003070F01000200EB54748029047480090474890
S3150800308002904748029047480090474802904748B0
S31508003090019047480290474802904748029047489F
S315080030A00290474801904748019047480190474891
S315080030B00290474801904748029047480190474880
S315080030C00190474801904748019047480290474871
S315080030D0029047480290474801904748029047485F
S315080030E00290474801904748019047480190474851
S315080030F00190474801904748019047480290474841
S31508003100029047480290474802904748019047482E
S31508003110019047480190474802904748029047481F
S315080031200290474801904748019047480190474810
S315080031300090474801904748029047480290474800
S3150800314002904748029047480290474802904748ED
S3150800315002904748019047480290474802904748DE
S3150800316001904748019047480290474802904748CF
S3150800317001904748019047480290474802904748BF
S315080031800190474801900298029001980190009892
S3150800319000900EBDF4580008585A0008F558000863
S315080031A0F6580008F8580008FC58000800590008A6
S315080031B0FD58000828590008295900082A59000806
S315080031C02C5900082E590008305900085059000893
S315080031D05259000854590008565900085859000809
S315080031E05A5900085C5900088C5900088D5900087E
S315080031F08E590008905900089259000893590008FA
S315080032009459000896590008985900089A590008D0
S315080032109C590008A0590008D0590008D15900083F
S31508003220D2590008D3590008D4590008D6590008BD
S31508003230D8590008005A0008015A0008025A00081E
S31508003240035A0008045A0008065A0008085A0008D3
S315080032500C5A00080D5A00080E5A00080F5A0008A2
S31508003260105A0008115A0008125A0008135A000882
S31508003270145A0008165A0008175A0008185A00085F
S315080032801A5A00081C5A00081D5A00081E5A000837
S31508003290205A0008505A0008515A0008525A000885
S315080032A0545A0008002400BF00BF00BF4020FDF7A5
S315080032B007F8044600BF00BF08480068401C0749D5
S315080032C0086007480068401C0549086000BF00BF41
S315080032D02046FDF703F800BFE6E70000841000204B
S315080032E0CC10002010B58AB0044600200E490860AC
S315080032F00B2000210591CDE90704069108460B49E4
S3150800330009680B4A12680B4B1B68CDE90132CDE9F7
S3150800331003101F200023084A08A100900C48FFF755
S3150800332053FB0AB010BD000084100020985800080E
S315080033309458000890580008A532000875432F4F86
S31508003340532D4949492049646C65205461736B00C3
S315080033505C2300200021034A1160034A1180018082
S31508003360704700009C100020A010002070B5014690
S315080033701A4D2D681DB945F21E750D8070BD184D84
S315080033802D881DB945F21D750D80F7E7134D286880
S315080033902A681032124D2D886D1EACB2002308E043
S315080033A00260002545600581C560103010325D1C3D
S315080033B0ABB2A342F4DB0025056045600581C56014
S315080033C0064D2D68074E3560054D2D88B5800025BC
S315080033D0F58035810D8000BFD0E70000B45800089D
S315080033E0AC5800082024002010B5014648894B89AE
S315080033F0BBB10A680B4B1B6813600A4C4B68236009
S315080034002346DB884C891B1B064CE38023469B8896
S315080034104C892344034CA38000234B818B810B608A
S315080034204B6010BD20240020018100224281828148
S31508003430026042607047000009A1C1610021416134
S315080034400849096811B90021816105E0054909683B
S3150800345081610449096848610249086070470000AB
S3150800346020000000A4100020026C0A620164704764
S315080034702DE9F84305462C6C25E0D4F82090FDF795
S3150800348047F98046C4F82C802146284600F034F8CF
S3150800349004F10806306820B9002084F82800606224
S315080034A010E037686562012084F82800214638460E
S315080034B0FFF7DAFF00231A4639462046CDF8008082
S315080034C000F0F6F84C46002CD7D1BDE8F88330B5A5
S315080034D004461F2004F140010AE00D68AB6823B1D9
S315080034E093F83B20824200DA10460D6805F1200168
S315080034F00D68002DF1D130BD024602F1400002E010
S31508003500036803F1200003688B42F9D103681B6A3C
S31508003510036070472DE9F04105460C4616461F46DE
S3150800352084F83860002084F839003946204600F0CF
S31508003530EDFB3DB105F1080865632146404600F0FC
S315080035405DF801E0002060632146284600F002F895
S31508003550BDE8F08110B540B14468C1F8C04000F13B
S3150800356008031A68D468C46113E091F83840022C3D
S3150800357002D0072C08D103E006A4C1F8C04007E032
S3150800358006A4C1F8C04003E007A4C1F8C04000BFC4
S3150800359000BF10BD5461736B205100005461736BFA
S315080035A02053656D000000002000000010B50A4693
S315080035B006A4C2F8C04040B100F10803196811B169
S315080035C0CC68C46101E001A4C46110BD20000000FC
S315080035D070B50446666B06F108052868C06A38B1F6
S315080035E0204600F03EF866632146284600F006F8B5
S315080035F070BD0021016041600181704710B591F8E6
S315080036003B3004683CB9012404810024CC620C6375
S315080036100160416024E00489641C0481026805E0B5
S3150800362092F83B409C4200DD02E0D26A002AF7D1BC
S3150800363000BF3AB90024CC6244680C630C6BE162A3
S3150800364041600DE0146B2CB9CA6200240C63116347
S31508003650016005E0CA62146B0C630C6BE1621163CE
S3150800366010BD10B5446B14B3446B04F108010C6823
S31508003670E46A1CB900240C604C6011E0046B24B9A0
S31508003680C26A002414630A600AE0C46A24B9036B98
S315080036900024DC624B6003E0036BC26ADA621363E0
S315080036A00C89641E0C810024C4620463446310BD43
S315080036B02DE9F04105460C4616461F46DDF81880EA
S315080036C094F83A00082845D2DFE800F0040508090E
S315080036D00607272800BF00BF00BF3CE000BF66669C
S315080036E0A4F86870C4F84C8015B12046FFF7B9FFF6
S315080036F021462846FFF75AFF94F83A00032802D1D4
S31508003700204600F005FD204600F068F80020383411
S31508003710A070607004F838091DE000BF6666A4F85A
S315080037206870C4F84C8015B12046FFF79AFF214609
S315080037302846FFF73BFF94F83A00072802D12046AF
S3150800374000F0E6FC04203834A0700020607004F80D
S31508003750380900E000BF00BFBDE8F08110B5034995
S315080037600868FCF7C8FDC0B210BD0000AC10002008
S31508003770002004E00021034A42F82010401C0028DB
S31508003780F8D07047AC10002004490968C0F11F033F
S3150800379001229A401143014A11607047AC1000207B
S315080037A004490968C0F11F0301229A409143014A5E
S315080037B011607047AC100020002109E001EB4102BE
S315080037C0054B03EB82000022028102604260491C1D
S315080037D02029F3D3704700002C24002010B5044696
S315080037E094F83B00FFF7D0FF94F83B0005490978A9
S315080037F0884203D1204600F027F802E0204600F070
S3150800380003F810BDAA10002010B590F83B3003EB62
S3150800381043030C4C04EB83010B683BB901230B8172
S315080038200023036143610860486009E00B895B1C5B
S315080038300B810B680361002343610A6850610860C5
S3150800384010BD00002C24002010B590F83B3003EB87
S3150800385043030B4C04EB83010B683BB901230B8133
S315080038600023036143610860486008E00B895B1C1C
S315080038700B81002303614A6842611061486010BDEC
S315080038802C2400202DE9F041054695F83B0000EB75
S315080038904000124901EB80046F692E6987B946B961
S315080038A0002020812060606095F83B00FFF778FFD4
S315080038B00EE02089401E208100207061266007E006
S315080038C02089401E20813E610EB9676000E077615D
S315080038D0002068612861BDE8F08100002C240020E2
S315080038E088B00020009006E0BD490968480002AA91
S315080038F00021FFF747FBBB4800780128F4D102A84E
S31508003900FEF7C8FF4FF00008B7480068B4490968D1
S31508003910884205D9B4480068B1490968B0FBF1F88E
S31508003920B8F1000F04D1B04800680A21B0FBF1F8DD
S3150800393000BFFCF7EDFE814600BF00BF4020FCF744
S31508003940BFFC009000BF00BFA8480068A8490860EF
S315080039500020A649086000BF00BF0098FCF7BEFC1F
S3150800396000BF00BFA3480068A1490968884248D932
S31508003970A0480068A049884205D242F21070049017
S315080039800120039023E09B4800689C49884205D2A1
S315080039904FF47A7004900A20039018E0954800685E
S315080039A09749884203D26420049003900FE0914817
S315080039B000689449884205D20A2004904FF47A7028
S315080039C0039004E00120049042F2107003908948A5
S315080039D001680398B1FBF0FB8549049809684843D8
S315080039E0B0FBFBF042F21071081A87490880874835
S315080039F000880988884207DA83480088834908804E
S31508003A0002E0002080490880FEF7DCFF002500BFA1
S31508003A1000BF4020FCF754FC009000BF00BF7C4864
S31508003A20046800BF00BF0098FCF758FC00BF00BF41
S31508003A3028E000BF00BF4020FCF742FC009000BF12
S31508003A4000BF54F8A00F6060002044F8A00900BF2A
S31508003A5000BF0098FCF742FC00BF00BFD4F8A400E2
S31508003A60054400BF00BF4020FCF72AFC009000BFB9
S31508003A7000BFD4F8BC4000BF00BF0098FCF72EFC7E
S31508003A8000BF00BF002CD4D15DB35B48854205D288
S31508003A9042F210700690012007901DE057488542B3
S31508003AA005D24FF47A7006900A20079014E054481D
S31508003AB0854203D26420069007900DE0514885425E
S31508003AC005D20A2006904FF47A70079004E0012088
S31508003AD0069042F2107007900798B5FBF0F0059033
S31508003AE003E0002006900120059000BF00BF40209B
S31508003AF0FCF7E6FB009000BF00BF4548046800BF1E
S31508003B0000BF0098FCF7EAFB00BF00BF2CE0D4F822
S31508003B10A400069948430599B0FBF1F086B242F233
S31508003B201070864200D90646A4F89060B4F8920050
S31508003B30B04201DAA4F8926002AB04F1B002111D9A
S31508003B402046FFF7F7F800BF00BF4020FCF7B8FB98
S31508003B50009000BF00BFD4F8BC4000BF00BF00986B
S31508003B60FCF7BCFB00BF00BF002CD0D100272948BA
S31508003B70D0F800A00AF1200A274800680838019002
S31508003B8002E00AF1040A7F1CDAF8000010B901986D
S31508003B908742F6D3214807601F480068C01B2049A2
S31508003BA0086020480078012805D100201D490870C2
S31508003BB002A8FEF76FFEFCF7ABFDA0EB09001A4959
S31508003BC008601A4800680968884203D216480068DF
S31508003BD01649086002AA00214046FFF7D3F9A8E66D
S31508003BE0BC580008D8100020D4580008CC10002073
S31508003BF0D4100020D0100020801A060000093D00CD
S31508003C00005A62020084D717C8100020CA10002084
S31508003C10E8100020A0580008A45800088C100020BE
S31508003C2090100020C6100020DC100020E0100020B4
S31508003C3010B58AB004460020214908602149086069
S31508003C4021490860214908702149087021490860FE
S31508003C50214908602148006820B946F62B60208073
S31508003C600AB010BD1E4800681E490968884203D27A
S31508003C7046F62C602080F3E71B4800781F2803D3FC
S31508003C8046F62A602080EBE7032000210591CDE95E
S31508003C9007040691084612490A68144909680F4B31
S31508003CA01B68CDE90131CDE903200F4800780023D0
S31508003CB00F4A10A100901448FEF786FE00BFCFE712
S31508003CC0CC100020D4100020D0100020D8100020DE
S31508003CD0C61000208C10002090100020C058000844
S31508003CE0C8580008D0580008B8580008C458000832
S31508003CF0E138000875432F4F532D4949492053741D
S31508003D006174205461736B00AC25002070B50446BD
S31508003D100D4655B12B46084800210268204600F09A
S31508003D205BF9032084F83A0002E0022084F83A009E
S31508003D302046FFF7A7FD70BDF01000202DE9F041E1
S31508003D4004460D4600BF002694F83B7094F83A00E6
S31508003D5008285DD2DFE800F004191E1F1A1B20216F
S31508003D602046FFF78FFD84F83B5094F83B00FFF799
S31508003D700BFD2B480068844203D12046FFF744FD1B
S31508003D8002E02046FFF760FD44E000BF00BF84F86C
S31508003D903B503FE000BF00BF00BF84F83B5094F89B
S31508003DA0380008282FD2DFE800F02E042F2E0A0547
S31508003DB0063000BF00BF2046FFF70AFC26E0204673
S31508003DC0FFF706FC606B466AAF4205DD96F83B00D6
S31508003DD0A84217DC002615E096F83B00B84211D138
S31508003DE03046FFF774FB054696F83C00A84202DA0F
S31508003DF096F83C0000E02846054696F83B00A8429F
S31508003E0000D1002602E000BF00BF00BF00BF01E0EE
S31508003E10BDE8F08100BF3446002C94D100BFF7E717
S31508003E20241100200021C0F8B8100949096819B9F9
S31508003E300021C0F8BC1007E005490968C0F8BC10A5
S31508003E4003490968C1F8B8000149086070470000CD
S31508003E50E8100020D0F8B820D0F8BC104AB90D4BAD
S31508003E60196011B10023C1F8B8300023C0F8BC307E
S31508003E700FE029B90023C2F8BC30C0F8B83008E012
S31508003E80C2F8BC10C1F8B8200023C0F8BC30C0F88E
S31508003E90B8307047E81000200021044A1160044A2F
S31508003EA01180044A1160018070470000E810002064
S31508003EB0EC100020E410002010B504460020206015
S31508003EC0A060606020616061A061E06122A0E0609E
S31508003ED0002020626062A062E0646066A4F8680060
S31508003EE0002104F16C00FFF79FFA00202C342065AE
S31508003EF06065A065A4F86000E0656062E067C4F8E4
S31508003F008000A06184F86200C4F88800C4F88400C0
S31508003F10A083A062E06220636063A4F86400A4F84A
S31508003F206600A066E066FCF7F3FB20670020606782
S31508003F3020606060A06020736073A0732020E07327
S31508003F40207400206061C4F88C00C4F8900004A0B6
S31508003F50C4F894002C3C10BD3F5461736B000000FC
S31508003F602000000008B504480068FEF7E2FE69462E
S31508003F700020FEF709FE08BD2411002010B50246F0
S31508003F800B46002107E0064C1068A04201D000202D
S31508003F9010BD121D491C0829F5D30120F8E70000B9
S31508003FA04523CDAB0246002003E0034B42F8203000
S31508003FB0401C0828F9D370474523CDAB0021018062
S31508003FC0034A1160034A11609180D180704700004E
S31508003FD0F0100020F41000202DE9F04304460F46A7
S31508003FE09446984608EB0C00DFF89090D9F80090B4
S31508003FF0B944A0EB09021AB900206065BDE8F08350
S315080040001F4B186838B962650020A061E0611C6022
S3150800401001209880F2E79888401C98801968486DB6
S31508004020C61BB2420BD2C86948B96265B01A486560
S315080040300020E061A161CC611C600120DEE7921BD3
S315080040400D46A96903E0486D121A0D46896911B132
S31508004050486D9042F7D949B1CD696265E561A161BC
S31508004060486D801A4865CC61AC6104E06265E5611B
S315080040700020A061AC610120C0E70000F01000201C
S31508004080F41000202DE9F04F06460C4691461F46CF
S315080040904FF0000BB9F1040F01D1002520E0B9F16A
S315080040A0080F1BD124B947F27E203880BDE8F08F6F
S315080040B0B56D16480068A0EB0508A0450AD3B8FBFD
S315080040C0F4F004FB0055B8FBF4F004FB108000B1D3
S315080040D02544B565B06D2044B06501E00B48056818
S315080040E023462A4659463046FFF776FF8246BAF1F6
S315080040F0010F05D1012086F83A000020388002E039
S3150800410047F27E20388000BFD0E70000F01000207C
S3150800411030B5C3698169134A9BB921B90024146073
S31508004120948044651CE00024CC614C6D456D2C449C
S315080041304C6511609488641E9480002484614465EB
S315080041400EE0996121B1CB614C6D456D2C444C65EF
S315080041500024C4619488641E9480002484614465A4
S3150800416030BD0000F410002010B5002400BF00BFC9
S315080041704020FCF7A5F8044600BF00BF08480949D7
S3150800418008600948086201F10800FFF732FA00BF23
S3150800419000BF2046FCF7A2F800BF00BF10BD000014
S315080041A0434F4E447026002094260020F8B500267A
S315080041B000BF00BF4020FCF783F8064600BF00BFDB
S315080041C0FCF7A6FA04460F48C4620F4D286838B9AA
S315080041D000BF00BF3046FCF781F800BF00BFF8BD3E
S315080041E000231A460949084808380094FFF760FA78
S315080041F000BF00BF3046FCF771F800BF00BF00BF24
S31508004200EDE700009426002078260020C42600202A
S315080042102DE9F84307464FF0000800BF00BF4020CD
S31508004220FCF74EF8804600BF00BFFCF771FA064659
S315080042303F48C66201463F48FFF75EF93C4D0835E0
S315080042403C4890F83B003B4991F83C1088420AD01C
S31508004250384890F83C00374981F83B00084690F802
S315080042603C0035490870286828B90020304948625A
S3150800427081F8280010E02C682D48446201202C495A
S3150800428081F828002046FFF7EFF800231A46214652
S3150800429027480096FFF70CFA3B460322254927488C
S315080042A0FFF738F900BF00BF4046FCF717F800BF14
S315080042B000BFFEF74BFA00BF00BF4020FCF700F82E
S315080042C0804600BF00BF1A48406A80B91849194895
S315080042D0FFF7CAF8174816494862012081F82800EE
S315080042E000BF00BF4046FBF7F9FF00BF1DE01048BE
S315080042F0446A94F83B000F4991F83B10884205DD63
S315080043000C4890F83B102046FFF718FD00230422BE
S3150800431008490748FFF7FEF800BF00BF4046FBF70D
S31508004320DDFF00BF00BFFEF711FABDE8F883000005
S3150800433094260020C4260020AA10002070260020FB
S3150800434010B58AB0044600202A4908802A49086020
S315080043502A4908602A4908802A4800682A490968BB
S31508004360B0FBF1F02949086000202949086029496D
S315080043700860224628A12C48FEF784F8208808B150
S315080043800AB010BDFFF7F0FE2848006818B947F2D2
S3150800439047302080F4E7264800682649096888429D
S315080043A003D247F248302080EAE7234800781F28DE
S315080043B003D347F246302080E2E70B20002105911F
S315080043C00A46CDE907040691194800681B49096899
S315080043D0164B1B68CDE90131CDE903021648007872
S315080043E00023174A17A100901C48FEF7EDFA00BFF4
S315080043F0C6E7000010110020041100200C1100204F
S3150800440008110020D4580008DC58000820110020A4
S3150800441014110020181100204F5320546D72204D9E
S31508004420757465780000000094260020E05800089E
S31508004430E8580008D0580008D8580008E45800087A
S315080044403145000875432F4F532D49494920546972
S315080044506D6572205461736B00000000C42600204D
S315080044602DE9F047054688462848006870B90020B7
S315080044702861686125480560012025490880254886
S31508004480C0F80080FFF792FEBDE8F0872048008854
S31508004490401C1F490880A86940441E490968461AF5
S315080044A01A480468D4F818904E4510D2606970B955
S315080044B0A9EB0600A061002068612C6165611348BC
S315080044C005601448C0F80080FFF770FEDCE7A6EB2D
S315080044D0090627463C6903E0A069361A2746246977
S315080044E014B1A069B042F7D94CB16769AE616F6182
S315080044F02C61A069801BA06165613D6104E0AE6125
S315080045006F61002028613D6100BFBDE70C110020E6
S31508004510081100201C1100201CB501A800231A460A
S31508004520194600900148FDF7FDFF1CBD94260020A2
S315080045304FF0000AFFF7F0FF00BF3D48006810B9CA
S315080045404FF0000903E03A480068D0F8189048464A
S31508004550FFF75EFE3648006800B9EEE7FCF7D8F8C4
S31508004560804600BF00BF4020FBF7AAFE824600BF78
S3150800457000BF3048076800BF00BF5046FBF7AEFED5
S3150800458000BF00BF2C4800683D1A2B480760284822
S3150800459004680CE0A069A84204D2A0692D1A00207C
S315080045A0A06103E0A069401BA061002524690DB144
S315080045B0002CEFD11E48046826E0042084F8260063
S315080045C0A66816B12046E168B04794F82600042884
S315080045D018D119480168204600F034F8A08C022842
S315080045E009D184F82600206AA0611348016820468C
S315080045F0FFF736FF06E0002060612061A061032016
S3150800460084F826000A48046814B1A0690028D4D0A2
S31508004610FCF77EF8A0EB080008490860084800681F
S315080046200968884203D2054800680549086084E796
S315080046300C110020F01000201C110020141100207D
S31508004640181100202DE9F04105460F46D5F81480CB
S315080046502C69B8F1000F40D154B9002029490860E7
S3150800466029490880A86129480760FFF79FFD46E0A9
S3150800467025480088401E24490880244800683E1AB8
S3150800468000206061A069A9690844A0611D4804600A
S315080046900EE0A069B04204D2A069361A0020A061D3
S315080046A003E0A069801BA0610026A046D8F8104048
S315080046B00EB1002CEDD1134800688069A9698842BB
S315080046C003D110480068806918B910480760FFF7D9
S315080046D06DFD00202861A86111E00B480088401E86
S315080046E009490880C8F810402CB1C4F81480A0699C
S315080046F0A9690844A061002068612861A861BDE82D
S31508004700F08100000C110020081100201C11002067
S315080047102DE9F04104460D4616460E4F00BF38787F
S3150800472008B900F0E3FB00BFEFF31180074620202D
S3150800473080F3118800BF00BF32462946204600F0A4
S315080047400BF88046F8B280F3118800BF00BF4046D8
S31508004750BDE8F081441600202DE9F0470746884653
S315080047601646C24607EB47011B4800EBC109D9F8B4
S31508004770140020B1012811D0022826D11EE048468F
S3150800478000F0ECFB0546B54201D2002405E03446AC
S3150800479032465146484600F038FD18E0484600F0D3
S315080047A0DDFB0546B54201D2284600E03046044600
S315080047B022465146484600F028FD08E03246514652
S315080047C0484600F0E7FC044601E0002400BF00BFAD
S315080047D02046BDE8F08700005C1600200FB438B507
S315080047E0044606A800906A462046059900F007F890
S315080047F0054600200090284638BC5DF814FB2DE9D4
S31508004800F04F99B082460D46144603A814904020EE
S31508004810159000201690CDF860A0179000BF2E784E
S315080048206D1C06B9DDE0252E79D100274FF0010968
S3150800483000BF2E78232E12D02B2E0CD02D2E02D070
S31508004840302E10D103E047F001076D1C0EE047F04B
S3150800485002076D1C0AE047F004076D1C06E047F0E6
S3150800486008076D1C02E04FF0000900BF00BFB9F150
S31508004870000FDED14FF0000800BF2E78302E01DB86
S31508004880392E00DD07E06D1CA6F1300008EB880123
S3150800489000EB4108F1E700BF002013902E782E2E7A
S315080048A012D16D1C00BF2E78302E01DB392E00DDAB
S315080048B009E06D1CA6F13000139901EB810100EBAC
S315080048C041001390EFE700BF2E7800BF6C2E01D091
S315080048D0682E02D16D1C2E7800E000E0F6E700BFD6
S315080048E0702E5DD008DC252E6AD0582E35D0632E62
S315080048F009D0642E69D113E0732E3CD0752E1DD0D5
S31508004900782E62D128E02168081D2060D1F8009031
S3150800491009F0FF0B594614A800F01AFC56E058E0B7
S315080049202168081D2060D1F80090CDE900870A2289
S31508004930494614A8139B00F01FFB47E02168081D91
S315080049402060D1F80090CDE900870A22494614A8CC
S31508004950139B00F087FB39E000BF2168081D206023
S31508004960D1F80090CDE900871022494614A8139B78
S3150800497000F078FB2AE02168081D2060D1F800B015
S3150800498000BF9BF800600BF1010B06B906E0314643
S3150800499014A800F0DDFB17980028F2DA00BF15E02E
S315080049A02168081D2060D1F80090002008210B46D8
S315080049B01022CDE90010494614A800F053FB05E083
S315080049C0252114A800F0C4FB00E000BF00BF6D1C41
S315080049D003E0314614A800F0BBFB17980028BFF681
S315080049E01EAF00BF179800280ADD169820B103A944
S315080049F05046169AFFF78CFEDDE916100844179004
S31508004A00179819B0BDE8F08F704700000348006892
S31508004A1040F47000014908607047000088ED00E026
S31508004A2070B50546AC6B0020E085E0842046FCF7AF
S31508004A30E6FF70BD0168C96821F490710268D1600B
S31508004A400168496921F0010102685161016B012978
S31508004A5005D10168C96821F010010268D1602021DA
S31508004A6080F83E1000210163704710B5044620689F
S31508004A70C06820F040002168C860202084F83D0006
S31508004A802046FDF789F9002010BD70B5044694F854
S31508004A903E00222856D1A068B0F5805F0CD1206967
S31508004AA050B90025A66A20684068C0F3080030801F
S31508004AB0A06A801CA06215E0A56A0026A068B0F569
S31508004AC0805F03D0A06828B9206918B920684068B3
S31508004AD0287004E02068406800F07F002870A06A0B
S31508004AE0401CA062E08D401E80B2E08540BB206875
S31508004AF0C06820F020002168C8602068C06820F4DB
S31508004B0080702168C8602068406920F0010021682B
S31508004B104861202084F83E00206B01280AD12068CD
S31508004B20C06820F010002168C860A18D2046FCF7F7
S31508004B3065FF02E02046FDF7F1F80020206370BD0E
S31508004B400020FCE70220FAE72DE9F84F0446206822
S31508004B50006920F44050E16808432168086121692A
S31508004B60A068084361690843E16908430090206822
S31508004B70C06849F20C618843009908432168C860F7
S31508004B802068406920F44070A1690843216848619B
S31508004B9076492068884203D075492068884203D13F
S31508004BA0FCF748FC814602E0FCF734FC8146E069E4
S31508004BB0B0F5004F6CD102206168A0FB0150034696
S31508004BC01920A9FB007001462A463846FBF79FFBC9
S31508004BD06421B0FBF1F04FEA001A02206168A0FBDD
S31508004BE001510B461920A9FB00712A463846FBF7E6
S31508004BF08EFB834602206168A0FB015003461920FC
S31508004C00A9FB00712A463846FBF781FB6421B0FBF5
S31508004C10F1F000EBC00101EB0010ABEB8000322194
S31508004C2001EBC0006421B0FBF1F000F0F8000AEBDC
S31508004C30400A02206168A0FB015003461920A9FB1F
S31508004C40007001462A463846FBF761FB8346022078
S31508004C506168A0FB015003461920A9FB00712A468A
S31508004C603846FBF754FB6421B0FBF1F000EBC001BA
S31508004C7001EB0010ABEB8000322101EBC000642190
S31508004C80B0FBF1F000F007005044216888606AE044
S31508004C9004206168A0FB015003461920A9FB007097
S31508004CA001462A463846FBF732FB824604206168ED
S31508004CB0A0FB015003461920A9FB007001462A46AD
S31508004CC03846FBF724FB6421B0FBF1F000EBC0018A
S31508004CD001EB0010AAEB8000322101EB00106421E1
S31508004CE0B0FBF1F000F0F00A04206168A0FB017047
S31508004CF003461920A9FB00513A462846FBF707FB4D
S31508004D006421B0FBF1F00AEB001A04206168A0FBED
S31508004D1001510B461920A9FB00712A463846FBF7B4
S31508004D20F6FA834604206168A0FB01500346192061
S31508004D30A9FB007001462A463846FBF7E8FA6421C3
S31508004D40B0FBF1F000EBC00101EB0010ABEB80000B
S31508004D50322101EB00106421B0FBF1F000F00F00E6
S31508004D60504421688860BDE8F88F000000100140B3
S31508004D700014014010B5034699629A85DA85002029
S31508004D801864222083F83E0000BF002083F83C0008
S31508004D9000BF1868C06840F480701C68E060186836
S31508004DA0406940F001001C6860611868C06840F0FE
S31508004DB020001C68E060002010BD014691F83D0007
S31508004DC0212828D18868B0F5805F0BD1086948B9D1
S31508004DD00A6A1088C0F308000B685860086A801CC5
S31508004DE0086205E00B6A581C086218780B68586058
S31508004DF0C88C401E80B2C88458B90868C06820F0BC
S31508004E0080000B68D8600868C06840F040000B68EE
S31508004E10D860002070470220FCE7000070B5002427
S31508004E202C4D2D48FCF7F6FD00BF03E0641CAC4290
S31508004E3000D904E02848FCF7E3FD2028F6D100BF96
S31508004E40002403E0641CAC4200D906E00122234991
S31508004E502148FCF741FF0028F4D100BF2048FCF7A1
S31508004E60D9FD002403E0641CAC4200D904E01C48C8
S31508004E70FCF7C6FD2028F6D100BF002403E0641C19
S31508004E80AC4200D906E0012214491548FCF724FF74
S31508004E900028F4D100BF1348FCF7BCFD002403E04A
S31508004EA0641CAC4200D904E00E48FCF7A9FD202892
S31508004EB0F6D100BF002403E0641CAC4200D906E02A
S31508004EC0012206490748FCF707FF0028F4D100BF6E
S31508004ED070BD0000FFFF0100F41100205E0E0020E7
S31508004EE0381200207C12002000BFFEE710B5124CD5
S31508004EF002202061606111A0A0611349E1614FF4AD
S31508004F00806121620021A1626162E1620BA0A06456
S31508004F100E49E164102121650021A1656165E165FD
S31508004F200BA1E01DFBF76AFA0AA12046FBF766FA11
S31508004F302020A07110BD0000441600205465726D33
S31508004F40696E616C00000000BC160020BC1A0020C7
S31508004F5052545400534547474552000010B5014680
S31508004F600A69CB689A4204D88C68641EE41AA018A9
S31508004F7001E0D41A601E10BD2DE9FC5F06460F46F7
S31508004F8092469846DDE90C45002F01DA784200E0A2
S31508004F90384683464FF0010903E09BFBFAFB09F10B
S31508004FA00109D345F9DAC84500D9C14634B1002FFD
S31508004FB003DB05F00400042800D1641E05F0020096
S31508004FC010B1B8F1000F11D005F0010070B96CB13D
S31508004FD008E0641E2021304600F0BAF8F068002880
S31508004FE000DA02E00CB1A145F3D300BFF06800284F
S31508004FF036DB002F05DA7F422D21304600F0A8F86F
S3150800500007E005F00400042803D12B21304600F000
S315080050109FF8F068002823DB05F00200022814D167
S3150800502005F0010088B9B8F1000F0ED16CB108E09F
S31508005030641E3021304600F08BF8F068002800DA4C
S3150800504002E00CB1A145F3D300BFF068002807DBE6
S315080050504346524639463046CDE9004500F002F847
S31508005060BDE8FC9F2DE9FC5F8046894615461E462D
S315080050700C9CCDF804900127BB4605E00198B0FBCF
S31508005080F5F001900BF1010B0198A842F6D25E45A6
S3150800509000D9B3460D9800F00100D0B9CCB10D98EF
S315080050A000F00200022803D116B93020009001E072
S315080050B02020009009E0641E4046009900F048F858
S315080050C0D8F80C00002800DA02E00CB1A345F2D3A8
S315080050D000BFD8F80C00002835DB09E0012E01D9FD
S315080050E0761E04E0B9FBF7FAAA4500D201E06F4341
S315080050F0F4E700BF00BFB9FBF7FA0AFB1799134894
S3150800510010F80A10404600F023F8D8F80C000028DA
S3150800511000DA03E0B7FBF5F7002FECD100BF0D98D6
S3150800512000F0010078B174B109E0641E2021404600
S3150800513000F00EF8D8F80C00002800DA02E00CB1EE
S31508005140A345F2D300BFBDE8FC9F000080580008C5
S3150800515070B504460E46A568681C6168814206D388
S3150800516020684655681CA060E068401CE060D4E9E9
S31508005170011088420DD1A26821682069FFF7C8FA94
S31508005180A168884203D04FF0FF30E06001E00020BC
S31508005190A06070BD2DE9F05F0446894617464FF0BA
S315080051A0000AE56800BFD4F81080A84503D9A8EB23
S315080051B00500461E04E0A5EB0800401CA1680E1A6F
S315080051C0A068401BB04201D9304601E0A068401BE8
S315080051D00646BE4201D2304600E0384606466068BA
S315080051E000EB050B324649465846FBF72BF9B24405
S315080051F0B144BF1B3544A068A84200D10025E5602C
S31508005200002FD0D15046BDE8F09F2DE9F04704465F
S3150800521089461546E668A068871BAF420AD96068C2
S3150800522000EB060A2A4649465046FBF70BF9701961
S31508005230E06014E0B846606800EB060A4246494654
S315080052405046FBF7FFF8A5EB0708D4F804A009EBCE
S31508005250070142465046FBF7F5F8C4F80C80BDE84E
S31508005260F087000002480068C0F30220704700007B
S315080052700CED00E010B5002804DB0A07130E054AFA
S31508005280135406E00A07140E034A00F00F031B1F07
S31508005290D45410BD00E400E018ED00E000BF7047EC
S315080052A070B58AB004460D4604B3208864281DDA12
S315080052B0208A0A21B0FBF1F609A8032100220592EB
S315080052C0CDE906210890208AE169CDE90116CDE9E4
S315080052D00302207A00902346064A29466068FDF7AD
S315080052E073FB2188044840F8214000BF38460AB0BD
S315080052F070BD0000B5570008901300202DE9F04155
S315080053008AB004460D4616461F46DDF840801C48FE
S315080053101C49086008464760C0F80880C4600661F2
S31508005320456100210176417681760121C176002109
S3150800533001774177FBF744FC18B101200AB0BDE8B4
S31508005340F08100200590069001200790002000902B
S315080053500190029003900490012008900E20099075
S3150800536069460848FBF7AEFA08B10220E6E70548A1
S31508005370FBF73AFD08B10320E0E70020DEE700006E
S3150800538000640040E815002070B504460D4600216B
S315080053900E48FBF729FB08B9002070BD2B460C4ABE
S315080053A000210A48FBF734FB08B10020F5E7084856
S315080053B00068A04205D10648806810B90448C0684C
S315080053C008B10020E9E70248007CE6E7E815002076
S315080053D028160020F8B504460D4616460027012073
S315080053E00090124804604460002010498860C86034
S315080053F0084606616B462A460D48FBF7B7F908B119
S315080054000120F8BD0AE0781C87B2B7F5805F05DB96
S3150800541007480099FBF77FF90120F2E70448FBF7F4
S31508005420B4FB0328EFD10020EBE70000101600209C
S31508005430E815002010B5044600204FF0E021086169
S315080054400420FCF7ADFA0148046010BD681000207E
S3150800545070B5034600224FF0E02675690D4E366892
S3150800546003FB06F44FF0E026B16910E04FF0E026A2
S31508005470B06988420BD0884202D20E1A324402E042
S315080054802E1A0E4432440146A24200D300E0EDE74C
S3150800549000BF70BD6810002010B50220FFF7D8FFC6
S315080054A010BD000000B587B000BF00BF0020019006
S315080054B01A48006840F00200184908600846006863
S315080054C000F00200019000BF00BF00BF00BF00BF90
S315080054D0002001900846006840F00200086008466F
S315080054E0006800F00200019000BF00BF00BF402026
S315080054F002900120039004900320059002A9084811
S31508005500FBF70AFD802002901120039002A90448A7
S31508005510FBF702FD00F006F807B000BD3038024080
S315080055200004024010B500BF002280210C48FBF79A
S31508005530F5FD00BFFFF7B0FF00BF01224021084874
S31508005540FBF7ECFD00BFFFF7A7FF00BF0122802194
S315080055500348FBF7E3FD00BFFFF79EFF10BD000001
S315080055600004024070B506460C460025304600F099
S315080055701DF80546A54203D2601B00F005F802E0B7
S31508005580012000F001F870BD38B504466A460021CE
S315080055902046FDF7F7FC38BD02460020914201D3AC
S315080055A0881A02E0C2F1FF335818704770B50446EE
S315080055B000F008F8064631462046FFF7EDFF054697
S315080055C0284670BD08B56846FDF73AFD08BD0000D7
S315080055D038B5FAF771FE00BFFFF7F4FF04460D4B26
S315080055E022460DA10020FFF7F9F80EA10020FFF7CB
S315080055F0F5F800BF6846FCF7F7FD0EA11248FFF75D
S315080056004FFE12A11648FFF74BFE6846FDF7F6F85F
S31508005610002038BD4258000825642025733E3E20E8
S3150800562000000000424D53207374617274200D0A05
S3150800563000000000706F6C6C5F73746172745F7445
S3150800564061736B3100000000080E0020706F6C6CEF
S315080056505F73746172745F7461736B32000000006B
S31508005660300E00201CB500BF13E0002005E0411CE9
S31508005670C9B20DF80010411CC8B20828F7DB082289
S3150800568069466620FFF7A6FE69466620FFF77CFE98
S3150800569000BFEAE738B5FBF753FD072302220821C6
S315080056A04FF4A87000F018F8A820FFF7C3FEFCF71F
S315080056B077FB4FF4E1342046FCF72EFC6005062301
S315080056C01A044FF4A00100900020FFF717FEFFF719
S315080056D0E9FE38BD00BFFEE72DE9F04192B08046ED
S315080056E00C4615461E460027302106A8FAF7EFFE97
S315080056F0142101A8FAF7EBFE00BF002000902A4803
S31508005700006840F08050284908600846006800F0A4
S315080057108050009000BF00BF00BF002000902348C3
S31508005720006840F48040214908600846006800F493
S315080057308040009000BF00BF01200690000407903B
S3150800574002200C9041050D91CDF83C800E941095E1
S31508005750119606A8FBF7D6FE07461FB1012012B020
S31508005760BDE8F0810F2001900220029000200390EE
S315080057704FF4A05004904FF480500590052101A8DD
S31508005780FBF780FD07460FB10120E8E7FBF7CCFCE5
S3150800579041F20101884205D10548006840F480704D
S315080057A0034908600020DAE74038024000700040EC
S315080057B0003C02402DE9F04105460026002D26D082
S315080057C02C46606908B16069804700BF00BFFFF7D3
S315080057D0F9FE07460F4B3A460FA10020FEF7FEFFDB
S315080057E0FFF7F0FE871B22883B460EA10020FEF736
S315080057F0F5FF00BFFFF7E6FE06460020E081608958
S31508005800A169884761893046FFF7ACFEDEE7BDE847
S31508005810F08100004758000825642025733E3E2085
S31508005820000000007461736B3A2564207065726924
S315080058306F643A25640D0A004FF04070E1EE100AD5
S3150800584070476D61696E007461736B5F74656D7026
S315080058506C617465006273705F7461736B5F626517
S3150800586061745F77646F6700000000000000000045
S3150800587001020304060708090000000001020304E8
S315080058803031323334353637383941424344454668
S31508005890CC1A0020060000004000000000010000AD
S315080058A0CC1B002080000000000200002000000041
S315080058B000020000CC1D00201E0000000A000000A7
S315080058C0CC1F00200A0000006400000090010000C0
S315080058D040000000E80300001D0000000A00000068
S315080058E05C2100200C00000080000000000200007F
S315080058F090080000010100007856341201010000EA
S315080059000000000000000000000000000000000089
S315080059100000000000000000000000000000000079
S31508005920000000000000000001010100280004003A
S315080059300000000000000000000000000000000059
S315080059400000000000000000000000000000000049
S3150800595001002000010010000C00100000000000EB
S315080059600000000000000000000000000000000029
S315080059700000000000000000000000000000000019
S315080059800000000000000000000000000101010006
S31508005990300001010C002000200004000400000073
S315080059A000000000000000000000000000000000E9
S315080059B000000000000000000000000000000000D9
S315080059C000000000000000000000000000000000C9
S315080059D00101010130000100000000000000000084
S315080059E000000000000000000000000000000000A9
S315080059F00000000000000000000000000000000099
S31508005A000101010128000C008001000004010101C8
S31508005A100101010100000101C400080001010000A4
S31508005A200000000000000000000000000000000068
S31508005A300000000000000000000000000000000058
S31508005A400000000000000000000000000000000048
S31508005A500101300050780000C10900007C5A000896
S31508005A60000000202C110000C4010008585B000843
S31508005A702C110020BC1A00002002000801FF01FFBB
S31508005A8001FF01FF01FF01FF01FF01FF01FF01FF08
S31508005A9001FF01FF01FF01FF011632011340061342
S31508005AA0200225F401D0071A90111395561B086594
S31508005AB004318220320213440D1320056BE80328B3
S31508005AC0411AD5288B040728A95811124C1A403AAE
S31508005AD04A402B2B024044C1C20C1A482C3C0C02EB
S31508005AE040392908D92DB92C3B10015849241908E1
S31508005AF00A19042C5D180240109029049A031829E3
S31508005B00B5091218195D0913180A12801829AC1953
S31508005B10800913180A1508181991091318199109F3
S31508005B2012782911F91829F8091218294829C17172
S31508005B30B91829C1E918196019BF09131819BF0935
S31508005B4010189C0802405FB918995F99A86119F363
S30D08005B5039A81103B124F40081
S7050800018968
